:020000040000FA
:04000000ABEF20F052
:08000800056ED8CF06F0E0CF31
:1000100007F00001E9CF0DF0EACF08F0E1CF09F0D9
:10002000E2CF0AF0D9CF0BF0DACF0CF0F3CF14F017
:10003000F4CF15F0FACF16F000C00FF001C010F0A9
:1000400002C011F003C012F004C013F0F2AA2CEFAA
:1000500000F0F2B4CFEF04F09DA032EF00F09EB0BC
:100060000DEF05F0F2A838EF00F0F2B28AEF07F0DA
:100070009DAA3EEF00F09EBA83EF07F00FC000F09C
:1000800010C001F011C002F012C003F013C004F060
:100090000DC0E9FF08C0EAFF088E09C0E1FF0AC0F1
:1000A000E2FF0BC0D9FF0CC0DAFF14C0F3FF15C08C
:1000B000F4FF16C0FAFF055007C0E0FF06C0D8FFE6
:1000C0001000F2CF0EF0F29EF76ADC0FF66E000E13
:1000D000F7220900F5500EBEF28E1200D04B896E49
:1000E000DAF7A517F8D8CC3B7623C11D539E5D39AE
:1000F000E0C203CFCD95CB1681AB0A8EFB63F9F43A
:10010000901011EE25C56F9704C068075F96436590
:10011000450F84BA579CCE1BA614B6A35CC677D5F0
:10012000B43D9827B9133A2D214018A028DEAC839E
:10013000E3DD696CB1B7492B9D0CC77109F57E826F
:100140006A78D2D71FA7F64C8BC3EF32E5A9377A6E
:10015000D41E7006558D52EC152059DBADBC7F4A7C
:10016000D6BBBEB03E7BBD79B894E12201C41C3140
:100170002E4F4D3675F0AFF28CE70D80196192E489
:10018000B3744635B212FE4E6D9BF1E951FF9FCA22
:100190006602AE0E93EA3C0854346264E691D37D65
:1001A0000BB5A41A5A86A12447DF8FE8883F443351
:1001B00060F34241EB2F9AEDFC48D1728A7356FAF4
:1001C000055E852A2C58E267FD7CA85B30D9385043
:1001D00087DC6BBFC9A29926AA29C800F2CF0EF00E
:1001E000F29EF76AF60FF66E010EF7220900F5503F
:1001F0000EBEF28E12004669726D776172652056EE
:10020000312E332E3120434320323030312D3230E5
:100210003038205261706861656C20416272616D96
:10022000732C207777772E746575746869732E63E5
:100230006F6D0000F2CF0EF0F29EF76A4E0FF66E71
:10024000020EF7220900F5500EBEF28E12007072F7
:100250006F626C656D20696E697469616C697A6939
:100260006E6720636172642C20676F696E6720740B
:100270006F20736C65657000F2CF0EF0F29EF76A26
:10028000920FF66E020EF7220900F5500EBEF28EA6
:10029000120070726F626C656D2072656164696EC8
:1002A000672042504200F2CF0EF0F29EF76AC00F74
:1002B000F66E020EF7220900F5500EBEF28E120005
:1002C00066696C652073797374656D20666F756EF1
:1002D0006400F2CF0EF0F29EF76AEC0FF66E020E9B
:1002E000F7220900F5500EBEF28E1200726F6F7485
:1002F000206469722073697A65206973202575000E
:10030000F2CF0EF0F29EF76A1A0FF66E030EF72286
:100310000900F5500EBEF28E120053504920746849
:10032000726F74746C653D2046415354212074688B
:100330006973206D6F646520646F6573206E6F74E0
:1003400020737570706F727420616C6C20636172C1
:1003500064732100F2CF0EF0F29EF76A6E0FF66E14
:10036000030EF7220900F5500EBEF28E1200535014
:1003700049207468726F74746C653D20534C4F57FC
:100380000000F2CF0EF0F29EF76A9C0FF66E030E9D
:10039000F7220900F5500EBEF28E12004D4F444573
:1003A0002069732053455249414C5F46554C4C5F80
:1003B0004E4F50494E00F2CF0EF0F29EF76AD00F2A
:1003C000F66E030EF7220900F5500EBEF28E1200F3
:1003D0004D4F44452069732050494E20544F2050C2
:1003E0004C415900F2CF0EF0F29EF76AFE0FF66E06
:1003F000030EF7220900F5500EBEF28E12004D4F8B
:10040000444520697320464F55522D464F555200A2
:10041000F2CF0EF0F29EF76A2A0FF66E040EF72264
:100420000900F5500EBEF28E12004D4F4445206972
:100430007320504152414C4C454C20504F52540077
:10044000F2CF0EF0F29EF76A5A0FF66E040EF72204
:100450000900F5500EBEF28E12004D4F4445206942
:10046000732053485546464C452F52414E444F4DFC
:100470000000F2CF0EF0F29EF76A8C0FF66E040EBB
:10048000F7220900F5500EBEF28E12004D4F444582
:100490002069732044454641554C5400F2CF0EF07C
:1004A000F29EF76AB60FF66E040EF7220900F550B9
:1004B0000EBEF28E1200666F6F6665726177203530
:1004C0000000F76AD20FF66E040EF7220900F5500D
:1004D00012005468697366696C65256C7500F2CF0B
:1004E0000EF0F29EF76AF80FF66E040EF72209007E
:1004F000F5500EBEF28E12006C6F73742061207383
:100500006563746F72210000F2CF0EF0F29EF76AFD
:10051000220FF66E050EF7220900F5500EBEF28E80
:1005200012005F736F6E672073746F707065642064
:10053000627920757365725F0000F2CF0EF0F29E53
:10054000F76A540FF66E050EF7220900F5500EBE3D
:10055000F28E1200736F6D6520696E666F206162A6
:100560006F757420636172643A00F2CF0EF0F29EF0
:10057000F76A840FF66E050EF7220900F5500EBEDD
:10058000F28E12002062706273743A25344C582047
:100590002000F2CF0EF0F29EF76AAC0FF66E050E59
:1005A000F7220900F5500EBEF28E12002042504292
:1005B0005F62707365633A25344C58202000F2CF97
:1005C0000EF0F29EF76AD80FF66E050EF7220900BC
:1005D000F5500EBEF28E1200204250425F5363501F
:1005E00065433A25344C58202000F2CF0EF0F29E9D
:1005F000F76A040FF66E060EF7220900F5500EBEDC
:10060000F28E1200204250425F527376645363436D
:10061000743A25344C5820200000F2CF0EF0F29EA0
:10062000F76A340FF66E060EF7220900F5500EBE7B
:10063000F28E1200204250425F4E6D4641543A25E0
:10064000344C58202000F2CF0EF0F29EF76A600F73
:10065000F66E060EF7220900F5500EBEF28E12005D
:100660002066617473746172743A2025344C58208A
:100670002000F2CF0EF0F29EF76A8C0FF66E060E97
:10068000F7220900F5500EBEF28E12002046697264
:10069000737444617461536563746F723A25344CAA
:1006A00058202000F2CF0EF0F29EF76ABE0FF66ED1
:1006B000060EF7220900F5500EBEF28E120070727F
:1006C0006F626C656D2072656164696E672066613A
:1006D00074207461626C652C207175697474696E24
:1006E0006720636861696E2E20536F7272792100F2
:1006F000F2CF0EF0F29EF76A0A0FF66E070EF7229F
:100700000900F5500EBEF28E1200565331303131D1
:100710003A20686172642072657365740000F2CFDC
:100720000EF0F29EF76A380FF66E070EF7220900F8
:10073000F5500EBEF28E1200200A0D00F2CF0EF020
:10074000F29EF76A560FF66E070EF7220900F55073
:100750000EBEF28E12004D4D432F534420696E6938
:10076000743A2053656E7420307834302028636DDD
:10077000643029205350490A0D00F2CF0EF0F29E4A
:10078000F76A940FF66E070EF7220900F5500EBEB9
:10079000F28E12004D4D432F534420696E69743A16
:1007A00020476F7420726573706F6E7365200A0D39
:1007B0000000F2CF0EF0F29EF76ACC0FF66E070E35
:1007C000F7220900F5500EBEF28E12005344206944
:1007D0006E69743A20636F6D6D616E6435352E2ECF
:1007E0002E00F2CF0EF0F29EF76AFC0FF66E070EA7
:1007F000F7220900F5500EBEF28E12006E6F7420C3
:10080000616E2053442C206D6179626520616E20F9
:100810006D6D633F0000F2CF0EF0F29EF76A300F6D
:10082000F66E080EF7220900F5500EBEF28E120089
:100830007965732C206974277320616E206D6D6358
:100840002100F2CF0EF0F29EF76A5C0FF66E080EF2
:10085000F7220900F5500EBEF28E12006661696C37
:100860006564206F7574206F662069646C652D2D3A
:100870002D00F2CF0EF0F29EF76A8C0FF66E080E86
:10088000F7220900F5500EBEF28E12004D4D432F97
:10089000534420696E69743A20476F74206F7574F1
:1008A000206F662069646C6520726573706F6E736B
:1008B00065200A0D0000F2CF0EF0F29EF76AD00F0D
:1008C000F66E080EF7220900F5500EBEF28E1200E9
:1008D0004D4D432F534420696E69743A20476F741D
:1008E0002073657420626C6F636B206C656E677437
:1008F0006820726573706F6E73652E20446F6E652D
:100900002E0A0D00F2CF0EF0F29EF76A1E0FF66E61
:10091000090EF7220900F5500EBEF28E1200492092
:10092000616D20746865204B696E67200000F2CF0E
:100930000EF0F29EF76A480FF66E090EF7220900D4
:10094000F5500EBEF28E12006F66204672616E6325
:1009500065210000F2CF0EF0F29EF76A6E0FF66E80
:10096000090EF7220900F5500EBEF28E12007768CC
:100970006F2061746500F2CF0EF0F29EF76A900F5F
:10098000F66E090EF7220900F5500EBEF28E120027
:10099000616C6C20746865207069653F2100300EC1
:1009A0000301DD6F0001DF5319E1E1AD05D04DC357
:1009B000DCF04DC3DDF012D083B408D0DC3D01D0B3
:1009C00001D0DC2BDD3D01D001D0DD2B83B606D07C
:1009D000DC5301E0DC07DD5301E0DD07DB5304E11C
:1009E0004DC3DCF04DC3DDF0DB2D06D083CFDCF052
:1009F000F00EDC17DCC0DDF0DB5105080BE1E1ADEA
:100A000005D04DC3DCF04DC3DDF004D083CFDCF066
:100A100083CFDDF0F2943EEF00F09E903EEF00F0C9
:100A20009EA8FED7AD6E000C006A016A026A036AD6
:100A30000301F96BFA6BFB6BFC6BF851F711F611C4
:100A4000F5112CE0200EFD6FD890F137F237F33717
:100A5000F437F937FA37FB37FC37F851FC5D08E11A
:100A6000F751FB5D05E1F651FA5D02E1F551F95DE3
:100A70000FE3F551F95FF651D8A0F63DFA5FF75153
:100A8000D8A0F73DFB5FF851D8A0F83DFC5FD880B7
:100A90000036013602360336FD2FD6D7030EEA6E36
:100AA000F90EE96E0001000CE9500301E96F3B0EFD
:100AB000F06F9A0EEF6FCA0EEE6FED6B0A0EEB6FD2
:100AC000E8C3F4F3E7C3F3F3E6C3F2F3E5C3F1F3EA
:100AD000F0C3F8F3EFC3F7F3EEC3F6F3EDC3F5F3AA
:100AE0000001A2DF0150EFCFE5F3ECCFE6F3ECCF4E
:100AF000E7F3ECCFE8F3005213E10301EB51010AF5
:100B0000D8A402D000010CD0E9510CE00F0BEB5D32
:100B100001E00EE2E9BF0CD0E9BD04D0200E03D005
:100B20000301E96B300E002600509EA8FED7AD6E83
:100B3000F0C3F4F3EFC3F3F3EEC3F2F3EDC3F1F359
:100B4000F86BF76BF66B0A0EF56F00016DDF03C0F3
:100B5000F0F302C0EFF301C0EEF300C0EDF30301C8
:100B6000EB2FAED70001000C0301EC6BED6B010E17
:100B7000EE6FDA6AD96A030EF16FE40EF06F030EBE
:100B8000EA6EE80EE96EF1C3E2FFF0C3E1FFEEC3E7
:100B9000EFF3D890E550EE02F350EC23F450ED2340
:100BA000EF2FF7D7ECC3DEFFEDC3ECF3ED6BD8B05E
:100BB000ED2BF02BD8B4F12BEE2BEE510508DFE135
:100BC0000001000CF29CF29EF2BEFDD79D9A9EAAF7
:100BD000FED7AECFDDF30301DD51000121DFDE5191
:100BE0006C0805E1DDC3DCF0300EDE6F85D1DE512F
:100BF000720805E1DDC3DDF0300EDE6F7DD1DE5120
:100C0000760807E1DDC3DDF0DDC3DCF0300EDE6F1A
:100C100073D1DE513008D8A46FD10301DD516C08C7
:100C200005E16C0E0001DE6F67D10301DD51720832
:100C300005E1720E0001DE6F5FD10301DD51760820
:100C400005E1760E0001DE6F57D10301DD51610829
:100C500006E10001E199300EDE6F4ED10301DD5156
:100C6000620806E10001E189300EDE6F45D1030123
:100C7000DD516B0808E10001E181E193300EDE6F88
:100C8000E19B3AD10301DD5174084AE19EAAFED7E7
:100C9000AECFDDF3DD510001C3DE0301DF6BDDC349
:100CA000DEF3DEC3DFF3DE6B9EAAFED7AECFDDF34D
:100CB000DD510001B5DE0301DD51DE27000EDF232B
:100CC000E36BE26BDFC3E1F3DEC3E0F30001E1813C
:100CD000E183E3C3F7F0E2C3F6F0E1C3F5F0E0C36C
:100CE000F4F00301E46BE451000161EC02F0030154
:100CF000E42B000195DE080E0301E45DF4E1410EF2
:100D0000E96EE3C3E8F3E2C3E7F3E1C3E6F3E0C36C
:100D1000E5F30001C9DEE19B300EDE6FEDD003018B
:100D2000DD516908D8A4E3D09EAAFED7AECFDDF38B
:100D3000DD51000175DE300E0301DD5FE36BE26B18
:100D4000E16BDDC3E0F3E3C3E7F3E2C3E6F3E1C342
:100D5000E5F3E0C3E4F3EB6BEA6BE96B0A0EE86FD3
:100D6000000102DF03C0E3F302C0E2F301C0E1F3DC
:100D700000C0E0F39EAAFED7AECFDDF30301DD5144
:100D800000014EDE300E0301DD5FDD51E027000E75
:100D9000E123E223E323E3C3E7F3E2C3E6F3E1C3A2
:100DA000E5F3E0C3E4F3EB6BEA6BE96B0A0EE86F83
:100DB0000001DADE03C0E3F302C0E2F301C0E1F3B5
:100DC00000C0E0F39EAAFED7AECFDDF30301DD51F4
:100DD000000126DE300E0301DD5FDD51E027000E4D
:100DE000E123E223E323E3C3E7F3E2C3E6F3E1C352
:100DF000E5F3E0C3E4F3EB6BEA6BE96B0A0EE86F33
:100E00000001B2DE03C0E3F302C0E2F301C0E1F38C
:100E100000C0E0F39EAAFED7AECFDDF30301DD51A3
:100E20000001FEDD300E0301DD5FDD51E027000E25
:100E3000E123E223E323E3C3E7F3E2C3E6F3E1C301
:100E4000E5F3E0C3E4F3EB6BEA6BE96B0A0EE86FE2
:100E500000018ADE03C0E3F302C0E2F301C0E1F364
:100E600000C0E0F39EAAFED7AECFDDF30301DD5153
:100E70000001D6DD300E0301DD5FDD51E027000EFD
:100E8000E123E223E323E35303E1E251000805E217
:100E9000E36BE26BFF0EE16FE06F0001E181E18344
:100EA000E3C3F7F0E2C3F6F0E1C3F5F0E0C3F4F01A
:100EB0000301E46BE451000161EC02F00301E42B57
:100EC0000001AEDD080E0301E45DF4E1410EE96EC0
:100ED000E3C3E8F3E2C3E7F3E1C3E6F3E0C3E5F31A
:100EE0000001E2DDE19B300EDE6F06D00301DD5133
:100EF000700803E10001E17B0301C00EF2129D8A3C
:100F0000000187EF07F0DB51060801E15BD69E9AEE
:100F10003EEF00F0DB51040814E184A00AD0740E07
:100F20007FDDF76BF66BF56B83CFF4F0E181E18346
:100F3000E18784B006D0760E73DD83CFDCF0DCC0B1
:100F4000DDF0DB2D0FD083506BDDF76BF66BF56BAF
:100F500083CFF4F00F0EF417F56BF66BF76BE181AE
:100F6000E183E187DB51050801E1E181F2923EEF87
:100F700000F0030EEA6ED10EE96EEF500EE00C0E9B
:100F8000016E006A002EFED7012EFBD7F70E006E11
:100F9000002EFED700D0EF2EF2D7000C03015D53D8
:100FA0002AE1040E5E6FC80ED16F0001E2DF03017B
:100FB0005E2FF9D75E6B5E510001A4DC03015E2B4E
:100FC00000012EDD0E0E03015E5DF5E15E6B5E51EC
:100FD0000001ADDC03015E2B000122DD0A0E0301DE
:100FE0005E5DF5E1020E5E6FC80ED16F0001C1DFDC
:100FF00003015E2FF9D75D2D3AD0040E5E6FC80E47
:10100000D16F0001B6DF03015E2FF9D7FE0E00019C
:1010100007DD010E05DDFE0E03DD020E01DD03011D
:101020005E6B5E51000196DC03015E2B0001F8DC73
:10103000070E03015E5DF5E1FE0E0001F1DCC00E5E
:10104000EFDC03015E6B5E51000195DC03015E2B5A
:101050000001E6DC0D0E03015E5DF5E1020E5E6F40
:10106000C80ED16F000185DF03015E2FF9D70001A3
:101070000DEF21F0020E03015D5F0CE3030EEA6E3B
:101080005D0EE96EEF5006E0020E006E002EFED7F8
:10109000EF2EFAD7000146EF21F00301896B070E0E
:1010A0008A6F8B96030E006E002EFED788C300F069
:1010B0008A51016E04E0D8900032012EFCD78B9843
:1010C00000B08B888B86210E006E002EFED782A08A
:1010D0000BD0010E006E8A51016E04E0D8900036EC
:1010E000012EFCD7005089138B96210E006E002E26
:1010F000FED78A518A07000AD9E189C301F00001AD
:10110000000CC66A8B828A8694988A9894967EC3CD
:1011100088F3C3DF7FC388F3C0DF030E0301856F4D
:10112000820E846F010E8425016E000E8521036EF0
:1011300001C086F3876F80C388F30001AEDF87C3E9
:10114000EAFF86C3E9FF01C0EFFF030E0301856FCD
:10115000820E85C303F0866F85C387F381C388F34E
:1011600000019BDF87C3EAFF86C3E9FF01C0EFFFF1
:101170008A8894884CC3C6FF030182C301F083C3ED
:1011800002F00001000C0301D451016AD35D03E2B7
:10119000D3C300F00CD0006A080ED56FD3370036E9
:1011A000D451005CD8B0006E0136D52FF7D70001BE
:1011B000000C0150D1C3D3F3640E0301D46F0001BE
:1011C000E2DF00C0D1F30150300E08E10301D2A3E9
:1011D0000ED0D2B70CD0D2B9200E04D00301D297D2
:1011E000D299D281012601509EA8FED7AD6ED1C3FF
:1011F000D3F30A0ED46F0001C6DF00C0D1F3015053
:10120000300E08E10301D2B70BD0D2A109D0D2B978
:10121000200E0001012601509EA8FED7AD6E0301ED
:10122000300ED127D1519EA8FED7AD6E0001000C23
:101230000301D06BD0510908D8A0DCD28B808B96EB
:101240001E0ED16F000195DEC78C220EC66E8B82FA
:101250008B901E0E0301D16F00018BDE0301CE6B5C
:10126000CE51090807E3C950FF0EC96EC730FEE32F
:10127000CE2BF6D78B92C950400EC96EC730FEE315
:10128000C950C96AC730FEE3C950C96AC730FEE316
:10129000C950C96AC730FEE3C950C96AC730FEE306
:1012A000C950950EC96EC730FEE3CD532EE0D16B09
:1012B000D15100018FEC03F0000907E00301D12BAD
:1012C0009EA8FED7AD6EF4D700010D0E9EA8FED7E6
:1012D000AD6E0A0E9EA8FED7AD6E0301D16BD15143
:1012E00000019EEC03F0000907E00301D12B9EA84A
:1012F000FED7AD6EF4D700010D0E9EA8FED7AD6EE1
:101300000A0E9EA8FED7AD6E0301010ED76F020E26
:10131000D96F080ED86FD85302E1D95312E0C950E3
:10132000FF0EC96EC730FEE3C9CFDAF3D751DA5DDD
:1013300003E1000E016E07D0D851D8B4D907D80701
:10134000EAD7010E016E0152D8A452D2CD5317E054
:10135000D16BD1510001BDEC03F0000907E003019E
:10136000D12B9EA8FED7AD6EF4D700010D0E9EA81E
:10137000FED7AD6E0A0E9EA8FED7AD6E0301CE6BF2
:10138000CF6BCD531EE00D0E000110EC05F00A0EE0
:1013900010EC05F00301D16BD1510001D9EC03F041
:1013A0000301D12B000110EC05F0150E0301D15DF6
:1013B000F3E10D0E000110EC05F00A0E10EC05F043
:1013C00003018B82C950FF0EC96EC730FEE3C950BE
:1013D000FF0EC96EC730FEE38B92C950770EC96EFF
:1013E000C730FEE3C950C96AC730FEE3C950C96AB5
:1013F000C730FEE3C950C96AC730FEE3C950C96AA5
:10140000C730FEE3C950F00EC96EC730FEE3800E50
:10141000D16F020ED36F080ED26FD25302E1D353B5
:1014200013E0C950FF0EC96EC730FEE3C9CFD4F335
:10143000D151D417D45303E1000E016E07D0D2511D
:10144000D8B4D307D207E9D7010E016E012C90D092
:10145000CE2BCE510A08D8B08AD0CF6BCD5316E030
:10146000D16BD1510001F1EC03F00301D12B00014C
:1014700010EC05F0180E0301D15DF3E10D0E000133
:1014800010EC05F00A0E10EC05F003018B82C95038
:10149000FF0EC96EC730FEE3C950FF0EC96EC730DC
:1014A000FEE38B92C950410EC96EC730FEE3C950AE
:1014B000C96AC730FEE3C950C96AC730FEE3C950E4
:1014C000C96AC730FEE3C950C96AC730FEE3C950D4
:1014D000FF0EC96EC730FEE3CF2BCD530CE02E0EAE
:1014E000000110EC05F0CFC3D1F31B0E0301D26F46
:1014F00000015FDE0301810ED16F020ED36F080E73
:10150000D26FD25302E1D35313E0C950FF0EC96E1C
:10151000C730FEE3C9CFD4F3D151D417D45303E17C
:10152000000E016E07D0D251D8B4D307D207E9D745
:10153000010E016E015219E1CD5316E0D16BD1516C
:1015400000010BEC04F00301D12B000110EC05F0BD
:10155000110E0301D15DF3E10D0E000110EC05F059
:101560000A0E10EC05F003018BD0CF3D8FD74FD77B
:10157000C950FF0EC96EC730FEE3C950FF0EC96ED9
:10158000C730FEE3C950FF0EC96EC730FEE3C95035
:10159000FF0EC96EC730FEE3C950690EC96EC73071
:1015A000FEE3C950C96AC730FEE3C950C96AC730F3
:1015B000FEE3C950C96AC730FEE3C950C96AC730E3
:1015C000FEE3C950FF0EC96EC730FEE3CE2BCD53EC
:1015D00018E02E0E000110EC05F02E0E10EC05F0B8
:1015E0002E0E10EC05F0CEC3D1F31B0E0301D26F0B
:1015F0000001DFDD640E10EC05F0200E10EC05F0AC
:101600000301810ED16F020ED36F080ED26FD25339
:1016100002E1D35313E0C950FF0EC96EC730FEE399
:10162000C9CFD4F3D151D417D45303E1000E016EC6
:1016300007D0D251D8B4D307D207E9D7010E016E33
:10164000015201E11DD0CE3D9CD6CD5316E0D16BA9
:10165000D151000121EC04F00301D12B000110EC69
:1016600005F0150E0301D15DF3E10D0E000110EC44
:1016700005F00A0E10EC05F00301010E016EBAD060
:10168000CD5325E00D0E000110EC05F00A0E10EC14
:1016900005F00301D16BD151000139EC04F00009D0
:1016A00007E00301D12B9EA8FED7AD6EF4D7000151
:1016B0000D0E9EA8FED7AD6E0A0E9EA8FED7AD6E8B
:1016C0000D0E10EC05F00A0E10EC05F003018B82F4
:1016D000C950FF0EC96EC730FEE3C950FF0EC96E78
:1016E000C730FEE3C950FF0EC96EC730FEE3C950D4
:1016F000FF0EC96EC730FEE38B92C950FF0EC96E54
:10170000C730FEE3C950500EC96EC730FEE3C95062
:10171000C96AC730FEE3C950C96AC730FEE3C95081
:10172000020EC96EC730FEE3C950C96AC730FEE376
:10173000C950FF0EC96EC730FEE3D76B020ED96FDA
:10174000080ED86FD85302E1D95312E0C950FF0EEA
:10175000C96EC730FEE3C9CFDAF3D751DA5D03E1D2
:10176000000E016E07D0D851D8B4D907D807EAD7F0
:10177000010E016E012C03D0010E016E3BD0C95049
:10178000FF0EC96EC730FEE3C950FF0EC96EC730E9
:10179000FEE38B82CD531DE0D16BD15100015BEC98
:1017A00004F0000907E00301D12B9EA8FED7AD6E1F
:1017B000F4D700010D0E9EA8FED7AD6E0A0E9EA8AE
:1017C000FED7AD6E0D0E10EC05F00A0E10EC05F014
:1017D0000301C950FF0EC96EC730FEE3C950FF0EAA
:1017E000C96EC730FEE34CC3C6FF000E016E02D0C7
:1017F000D02B20D50001000C0301D16BD151090879
:10180000D8A0CFD04CC3C6FFD0C3D6F3CFC3D5F337
:10181000CEC3D4F3CDC3D3F30001E2530DE1D8908E
:10182000D5C3D6F3D4C3D5F3D3C3D4F30301D36B59
:10183000D437D537D6370001C950FF0EC96EC7302F
:10184000FEE3C950FF0EC96EC730FEE38B92C9504C
:10185000510EC96EC730FEE3030E0301D86FD30EDD
:10186000D76F030ED725016E000ED821036E01C07D
:10187000E9FFEA6EEFCFD9F3C950D9C3C9FFC7302A
:10188000FEE3030ED86FD30ED76F020ED725016E7D
:10189000000ED821036E01C0E9FFEA6EEFCFD9F345
:1018A000C950D9C3C9FFC730FEE3030ED86FD30EAA
:1018B000D76F010ED725016E000ED821036E01C02F
:1018C000E9FFEA6EEFCFD9F3C950D9C3C9FFC730DA
:1018D000FEE3C950C96AC730FEE3C950FF0EC96EA6
:1018E000C730FEE3D76B020ED96F080ED86FD853FE
:1018F00002E1D95312E0C950FF0EC96EC730FEE3B2
:10190000C9CFDAF3D751DA5D03E1000E016E07D0DB
:10191000D851D8B4D907D807EAD7010E016E0152C1
:1019200033E1FE0ED76F020ED96F080ED86FD85371
:1019300002E1D95312E0C950FF0EC96EC730FEE371
:10194000C9CFDAF3D751DA5D03E1000E016E07D09B
:10195000D851D8B4D907D807EAD7010E016E015281
:1019600003E1000E016E1FD0D26BD23D01D00CD02E
:10197000C950FF0EC96EC730FEE3C950FF0EC96ED5
:10198000C730FEE3D22BF1D78B82C950FF0EC96E50
:10199000C730FEE3C950FF0EC96EC730FEE3D12B3E
:1019A0002DD7010E016E0001000C0301CE530CE097
:1019B000C950FF0EC96EC730FEE3C950FF0EC96E95
:1019C000C730FEE3CE07F2D70001000CC950FF0E6E
:1019D000C96EC730FEE3C9CF19F0C950FF0EC96EFA
:1019E000C730FEE3C9CF1AF0000CC950FF0EC96E14
:1019F000C730FEE3C950FF0EC96EC730FEE38B82CD
:101A0000C950FF0EC96EC730FEE3C950FF0EC96E44
:101A1000C730FEE3000C030164BF10D00F0E006E50
:101A2000633900160A0E005C03E2300E002602D075
:101A30006451002600509EA8FED7AD6E0F0E6317AE
:101A40000A0E635D02E2300E02D0649F6451632788
:101A500063519EA8FED7AD6E0001000CE56BE46BF0
:101A60000301D06BCF6BCE6BCD6B0001C5DEE30EF7
:101A70000301CE6F000199DFA9DF1AC0E5F0000174
:101A8000E46B1950E427000EE5231B0E0301CE6F13
:101A900000018BDFAADF0301646B636BE5C062F3B7
:101AA000E4C061F364C3D0F363C3CFF3E5C0CEF306
:101AB000E4C0CDF30001A0DE050E0301CE6F0001EE
:101AC00074DF84DFEB6B1AC0EAF080DF000E0001E8
:101AD000EA271950EB231AC0E3F078DF0301636BA8
:101AE000195063250001E86F000E03011A20000160
:101AF000E96F6CDF19C01CF169DF68DF67DF060E74
:101B00000301CE6F000151DF61DF0101176B166B1E
:101B1000156B146B0301636B626B63C303F062C3E9
:101B200002F0006A005019240101146F000E1A20FF
:101B3000156F000E0220166F000E0320176F17C1DD
:101B400060F316C15FF315C15EF314C15DF30001CC
:101B50003DDF0301636B626B63C303F062C302F09A
:101B6000006A005019240101146F000E1A20156F2D
:101B7000000E0220166F000E0320176F15C117F11B
:101B800014C116F1146B156B03015D51010114278B
:101B900003015E510101152303015F510101162369
:101BA0000301605101011723000110DF0FDF0EDF79
:101BB0000301636B626B63C303F062C302F0006AEC
:101BC000005019240101186F000E1A20196F000E21
:101BD00002201A6F000E03201B6F1BC160F31AC195
:101BE0005FF319C15EF318C15DF30001EFDEE70E8C
:101BF0000301CE6F0001D9DEF8DE0301636B626B77
:101C000063C303F062C302F0006A005019240101AB
:101C1000186F000E1A20196F000E02201A6F000EA6
:101C200003201B6F19C11BF118C11AF1186B196B36
:101C300003015D510101182703015E5101011923C0
:101C400003015F5101011A230301605101011B23AC
:101C50001BC10BF11AC10AF119C109F118C108F130
:101C60000001E851E425F86FE951E521F96FFA6BBD
:101C7000FB6B186AF2BE188EF29E0301E76BE66BEF
:101C8000E56B1CC1E4F317C1EBF316C1EAF315C110
:101C9000E9F314C1E8F30001B4EC05F018BEF28ECC
:101CA0000050E825E66F0150E921E76F0301646BFE
:101CB000636BE5C062F3E4C061F3E6C000F0026A62
:101CC000036A005061250001FC6FE75103016221A6
:101CD0000001FD6F0250030163210001FE6F0350FC
:101CE000030164210001FF6F0D0E10EC05F00A0ED8
:101CF00010EC05F00301616B615100019DEC02F0F5
:101D00000301612B000110EC05F0150E0301615D6C
:101D1000F3E10D0E000110EC05F00A0E10EC05F0D9
:101D20000301616B61510001B5EC02F00301612B0D
:101D3000000110EC05F0070E0301615DF3E1E5C061
:101D400063F3370E646F000166DEE4C063F3370EA1
:101D50000301646F00015FDE200E10EC05F0200E21
:101D600010EC05F00D0E10EC05F00A0E10EC05F06D
:101D70000301616B61510001C9EC02F00301612BA9
:101D8000000110EC05F00B0E0301615DF3E1EBC007
:101D900063F3370E646F00013EDEEAC063F3370E73
:101DA0000301646F000137DE200E10EC05F0200EF9
:101DB00010EC05F00D0E10EC05F00A0E10EC05F01D
:101DC0000301616B61510001DFEC02F00301612B43
:101DD000000110EC05F00B0E0301615DF3E1020E52
:101DE000626F300E000110EC05F00301622FF9D78D
:101DF000E3C063F3370E646F00010DDE200E10ECBC
:101E000005F0200E10EC05F00D0E10EC05F00A0E9A
:101E100010EC05F00301616B61510001F5EC02F07B
:101E20000301612B000110EC05F00E0E0301615D52
:101E3000F3E1E9C063F3370E646F0001ECDDE8C045
:101E400063F3370E0301646F0001E5DD200E10EC33
:101E500005F0200E10EC05F00D0E10EC05F00A0E4A
:101E600010EC05F00301616B615100010DEC03F012
:101E70000301612B000110EC05F00B0E0301615D05
:101E8000F3E1020E626F300E000110EC05F0030169
:101E9000622FF9D71CC163F3370E646F0001BBDDFD
:101EA000200E10EC05F0200E10EC05F00D0E10ECDD
:101EB00005F00A0E10EC05F00301616B61510001A1
:101EC00023EC03F00301612B000110EC05F00B0E75
:101ED0000301615DF3E1F9C063F3370E646F000144
:101EE0009ADDF8C063F3370E0301646F000193DDE0
:101EF000200E10EC05F0200E10EC05F00D0E10EC8D
:101F000005F00A0E10EC05F00301616B6151000150
:101F100039EC03F00301612B000110EC05F0110E08
:101F20000301615DF3E1E7C063F3370E646F000105
:101F300072DDE6C063F3370E0301646F00016BDDF1
:101F4000200E10EC05F0200E10EC05F00D0E10EC3C
:101F500005F00A0E10EC05F0000C0301C76BC66B10
:101F6000D890C237C337C437C537030ECE6FC20E01
:101F7000E96ECEC3EAFFEFCFCCF3C3C3C2F3C4C351
:101F8000C3F3C5C3C4F3C56B0001F8510301C227F5
:101F90000001F9510301C3230001FA510301C423D5
:101FA0000001FB510301C523C5C3D0F3C4C3CFF364
:101FB000C3C3CEF3C2C3CDF300011EDC012C4DD050
:101FC0005E0E10EC05F0C5C3D0F3C4C3CFF3C3C39A
:101FD000CEF3C2C3CDF310DC012C3FD0260E10ECA3
:101FE00005F00301CD6B000118EC09F0C5C3D0F377
:101FF000C4C3CFF3C3C3CEF3C2C3CDF3FCEC0BF029
:10200000012C2BD02A0E10EC05F00301CD6B000142
:1020100018EC09F0C5C3D0F3C4C3CFF3C3C3CEF3E8
:10202000C2C3CDF3FCEC0BF0012C17D00301CD6B38
:10203000CD51000152EC03F00301CD2B000110EC57
:1020400005F0310E0301CD5DF3E1FF0E006E016E70
:10205000026E036E43D00001E181CCC3CEF3A5DC58
:10206000B5DC0301CF6B036A1950CF25C66F03504F
:102070001A20C76F0001AADC0301CB6BCA6BC96BC6
:10208000C86BCF6B036A1950CF25C86F03501A2055
:10209000C96FCA6BCB6BC9C3CBF3C8C3CAF3C86BD8
:1020A000C96B026A036AC651C827C751C9230250C7
:1020B000CA230350CB23FF0ED880CC55CD6FCE6FF3
:1020C000000173DC83DC82DC90DCC8C300F0C9C390
:1020D00001F0CAC302F0CBC303F003010001000CFE
:1020E0001BC10BF11AC10AF119C109F118C108F19C
:1020F0000301606B5F6B5E6B5D6B0BC10FF10AC11F
:102100000EF109C10DF108C10CF10FC1C5F30EC1EB
:10211000C4F30DC1C3F30CC1C2F300011EDF03C041
:102120000BF102C00AF101C009F100C008F108C1B9
:1021300061F309C162F30AC163F301010B510F0B93
:102140000301646F010E5D27D8B05E2BD8B45F2BFE
:10215000D8B4602B64510F080CE3CFE16351FF0842
:1021600008E3CBE16251FF0804E3C7E16151EE08E7
:10217000C4E2186AF2BE188EF29E60C3E7F35FC332
:10218000E6F35EC3E5F35DC3E4F3EB6BEA6BE96B87
:10219000E3C0E8F30001B4EC05F018BEF28E03C012
:1021A00013F102C012F101C011F100C010F10101E0
:1021B00010371137123713371037113712371337DB
:1021C00010371137123713371037113712371337CB
:1021D000F00E1017FF0E1027D8A01127D8A0122735
:1021E000D8A0132700013CEF22F0110EC26E0A0E98
:1021F000C16E3E0EC06EC282C2A201D0FDD7C4CF56
:102200004DF303014D5302E1010E4D6F0001000C2F
:10221000016A026A006A036A0301C55102E1C451FE
:1022200018E0100EC66FD890C237C3370036033699
:10223000C551035C02E1C451005C07E3C451005E78
:10224000D8A00306C551035ED88001360236C62FDA
:10225000EAD70001000C03018B6B60C3C3F35FC3BB
:10226000C2F3270EC56F100EC46F0001D1DF01C08D
:102270006CF303018F6B8E6B8D6B6CC38CF3186AE0
:10228000F2BE188EF29E8FC3E7F38EC3E6F38DC3C2
:10229000E5F36CC3E4F3EB6BEA6B270EE96F100E0A
:1022A000E86F0001B4EC05F018BEF28E03C07AF3BB
:1022B00002C079F301C078F300C077F303017751CE
:1022C0005F5D8C6F785160598D6F000E79558E6F00
:1022D000000E7A558F6F186AF2BE188EF29EF46F58
:1022E0008EC3F3F38DC3F2F38CC3F1F3F86BF76B8A
:1022F000030EF66FE80EF56F000114EC05F018BE42
:10230000F28E00C06BF303018F6B8E6B8D6B6BC312
:102310008CF3186AF2BE188EF29E8FC3E7F38EC359
:10232000E6F38DC3E5F36BC3E4F3EB6BEA6B030EEB
:10233000E96FE80EE86F0001B4EC05F018BEF28E0C
:10234000005003017727015078230250792303506E
:102350007A2377515F5D8C6F785160598D6F000ED5
:1023600079558E6F000E7A558F6F186AF2BE188EEF
:10237000F29EF46F8EC3F3F38DC3F2F38CC3F1F3CB
:10238000F86BF76BF66B640EF56F000114EC05F05B
:1023900018BEF28E00C067F303018F6B8E6B8D6BDE
:1023A00067C38CF3186AF2BE188EF29E8FC3E7F3F0
:1023B0008EC3E6F38DC3E5F367C3E4F3EB6BEA6B1F
:1023C000E96B640EE86F0001B4EC05F018BEF28E04
:1023D00000500301772701507823025079230350DE
:1023E0007A2377515F5D8C6F785160598D6F000E45
:1023F00079558E6F000E7A558F6F186AF2BE188E5F
:10240000F29EF46F8EC3F3F38DC3F2F38CC3F1F33A
:10241000F86BF76BF66B0A0EF56F000114EC05F024
:1024200018BEF28E00C066F303018F6B8E6B8D6B4E
:1024300066C38CF3186AF2BE188EF29E8FC3E7F360
:102440008EC3E6F38DC3E5F366C3E4F3EB6BEA6B8F
:10245000E96B0A0EE86F0001B4EC05F018BEF28ECD
:10246000005003017727015078230250792303504D
:102470007A2377515F5D656F8A6B896B886B876B99
:102480001BC10BF11AC10AF119C109F118C108F1F8
:102490008A31826F8931816F8831806F87317F6F98
:1024A0008233813380337F338233813380337F3390
:1024B0008233813380337F330F0E821782C386F3DA
:1024C00081C385F380C384F37FC383F3186AF2BEAC
:1024D000188EF29E82C3F4F381C3F3F380C3F2F348
:1024E0007FC3F1F3F86BF76BF66BE3C0F5F3000114
:1024F00014EC05F018BEF28E03C082F302C081F323
:1025000001C080F300C07FF3186AF2BE188EF29EFD
:1025100082C3E7F381C3E6F380C3E5F37FC3E4F34B
:102520000301EB6BEA6BE96BE3C0E8F30001B4EC89
:1025300005F018BEF28E03C07EF302C07DF301C029
:102540007CF300C07BF303017B51835D7B6F7C5187
:1025500084597C6F7D5185597D6F7E5186597E6F80
:102560007F5306E1805304E1815302E1825324E06A
:102570000BC10FF10AC10EF109C10DF108C10CF137
:102580000FC1C5F30EC1C4F30DC1C3F30CC1C2F337
:102590000001E3DC03C00BF102C00AF101C009F144
:1025A00000C008F1FF0E03017F27D8A08027D8A024
:1025B0008127D8A08227D4D7020E0101085D03012C
:1025C0006F6F000E010109590301706F000E0101C8
:1025D0000A590301716F000E01010B590301726F5B
:1025E000E3C000F0016A026A036A03C08FF302C00D
:1025F0008EF301C08DF3E3C08CF3186AF2BE188E1F
:10260000F29E72C3E7F371C3E6F370C3E5F36FC3E1
:10261000E4F303C0EBF302C0EAF301C0E9F3E3C063
:10262000E8F30001B4EC05F018BEF28E03C072F3BB
:1026300002C071F301C070F300C06FF3FC510301DD
:102640006F270001FD51030170230001FE510301BA
:1026500071230001FF51030172237B516F277C51CD
:1026600070237D5171237E51722372C3D0F371C3E5
:10267000CFF370C3CEF36FC3CDF30001FCEC0BF0CE
:10268000100E0301646F6453D8B49CD00001E6ECD3
:102690000CF003018B2B195203E01950E50809E1F6
:1026A0000F0ECE6F0001D5EC0CF00F0E03018B273F
:1026B0007FD0300E195C6E6F300E1A5C6D6F0001AA
:1026C000E6EC0CF003018B2B300E195C6A6F300EB8
:1026D0001A5C696F0001E6EC0CF003018B2B300EE5
:1026E000195C686F6D516B5D57E16E516C5D54E123
:1026F0006851655D51E16951665D4EE16A51675D02
:102700004BE10001E6EC0CF0E6EC0CF019C061F3D3
:102710001AC062F3E6EC0CF0030E03018B2719C01C
:1027200063F361516D0809E061514D0806E06151A4
:10273000570803E0615177080FE16251500809E042
:102740006251700806E06251410803E0625161087D
:1027500003E16351330806E06351560803E0635117
:10276000760819E1000ED8808B558C6F010ED8A029
:10277000E8068D6F8CC3CEF30001D5EC0CF0F5ECC0
:102780000CF087C300F088C301F089C302F08AC34C
:1027900003F064D0030106D0030ECE6F0001D5EC28
:1027A0000CF003010A0ECE6F0001D5EC0CF0030112
:1027B000010E8727D8B0882BD8B4892BD8B48A2BA0
:1027C000640761D708C173F309C174F30AC175F3D3
:1027D00001010B510F0B0301766F0001F5EC0CF0BA
:1027E00003018A510101135D30E311E103018951B5
:1027F0000101125D2AE30BE1030188510101115D22
:1028000024E305E1030187510101105D1EE303018B
:1028100076510F08D8B002D0010117D0D8A430D615
:102820007551FF08D8B002D001010FD0D8A428D626
:102830007451FF08D8B002D0010107D0D8A420D627
:102840007351EF08D8B01CD6010100002D0E000115
:1028500010EC05F0006A016A026A036A000C0301C9
:10286000C251C403F3CF01F0F4CF00F0C503F3501D
:102870000026C351C403F3500020026E000182EF12
:1028800014F00301C16BBA6BB96BB86BB76B1BC1AA
:102890000BF11AC10AF119C109F118C108F164312B
:1028A000036E6331026E6231016E6131006E03327C
:1028B000023201320032033202320132003203327C
:1028C00002320132003200C0BDF301C0BEF3BEC30C
:1028D000C0F3BDC3BFF3BEC3C3F3BDC3C2F3C56B77
:1028E000E3C0C4F3000194DC02C0BEF301C0BDF339
:1028F000BEC3C3F3BDC3C2F30301C56BE3C0C4F3DE
:102900000001ADD702C0BCF301C0BBF30301BB5152
:10291000BF5DBB6FBC51C059BC6FBD5302E1BE531C
:102920002BE00BC10FF10AC10EF109C10DF108C175
:102930000CF10FC1C5F30EC1C4F30DC1C3F30CC13B
:10294000C2F30001ADEC0FF003C00BF102C00AF1BD
:1029500001C009F100C008F108C1B7F309C1B8F31B
:102960000AC1B9F301010B510F0B0301BA6FBD513D
:10297000D8B4BE07BD07D1D7BA510E0813E2FF0A7B
:102980000DE1B951FE080EE2FF0A08E1B851FE0858
:1029900009E2FF0A03E1B751EF0804E2020E016EFB
:1029A000DEEF18F0020E0101085D0301B36F000EA7
:1029B000010109590301B46F000E01010A59030115
:1029C000B56F000E01010B590301B66FE3C000F0B3
:1029D000016A026A036A03C0C5F302C0C4F301C0FE
:1029E000C3F3E3C0C2F3186AF2BE188EF29EB6C3F8
:1029F000E7F3B5C3E6F3B4C3E5F3B3C3E4F303C04D
:102A0000EBF302C0EAF301C0E9F3E3C0E8F300012D
:102A1000B4EC05F018BEF28E03C0B6F302C0B5F3F5
:102A200001C0B4F300C0B3F3FC510301B3270001AC
:102A3000FD510301B4230001FE510301B523000140
:102A4000FF510301B623026A036ABB51B327BC518D
:102A5000B4230250B5230350B623B6C3D0F3B5C395
:102A6000CFF3B4C3CEF3B3C3CDF30001FCEC0BF052
:102A7000030161510F0BC26FC36BC46BC56BC235D1
:102A8000006EC335016EC435026EC535036E003667
:102A9000013602360336003601360236033600367A
:102AA000013602360336F00E001600C0C1F3C1C372
:102AB000CEF30001D5EC0CF00301A86BA8511F0860
:102AC000D8A000D10001E6EC0CF00301C12B036A91
:102AD000A851BB0F016E000E032203C0C3F3036AAB
:102AE000A8519B0FE96E000E0320EA6EEFCFC4F3EE
:102AF000C3C3EAFF01C0E9FFC4C3EFFF036AA851E3
:102B00009B0F016E000E032203C0C3F3036AA8519A
:102B10007B0FE96E000E0320EA6EEFCFC4F3C3C350
:102B2000EAFF01C0E9FFC4C3EFFF036AA8517B0FAE
:102B3000016E000E032203C0C3F3036AA8515B0FAA
:102B4000E96E000E0320EA6EEFCFC4F3C3C3EAFFC1
:102B500001C0E9FFC4C3EFFF036AA8515B0F016E18
:102B6000000E032203C0C3F3036AA8513B0FE96EB2
:102B7000000E0320EA6EEFCFC4F3C3C3EAFF01C027
:102B8000E9FFC4C3EFFF036AA8513B0F016E000EBB
:102B9000032203C0C3F3036AA8511B0FE96E000EA2
:102BA0000320EA6EEFCFC4F3C3C3EAFF01C0E9FF1D
:102BB000C4C3EFFF036AA8511B0FE96E000E032088
:102BC000EA6E19C0EFFFA82B036AA851BB0F016E74
:102BD000000E032203C0C3F3036AA8519B0FE96EE2
:102BE000000E0320EA6EEFCFC4F3C3C3EAFF01C0B7
:102BF000E9FFC4C3EFFF036AA8519B0F016E000EEB
:102C0000032203C0C3F3036AA8517B0FE96E000ED1
:102C10000320EA6EEFCFC4F3C3C3EAFF01C0E9FFAC
:102C2000C4C3EFFF036AA8517B0F016E000E03229D
:102C300003C0C3F3036AA8515B0FE96E000E0320C3
:102C4000EA6EEFCFC4F3C3C3EAFF01C0E9FFC4C318
:102C5000EFFF036AA8515B0F016E000E032203C051
:102C6000C3F3036AA8513B0FE96E000E0320EA6E1E
:102C7000EFCFC4F3C3C3EAFF01C0E9FFC4C3EFFF52
:102C8000036AA8513B0F016E000E032203C0C3F379
:102C9000036AA8511B0FE96E000E0320EA6EEFCF06
:102CA000C4F3C3C3EAFF01C0E9FFC4C3EFFF036A73
:102CB000A8511B0FE96E000E0320EA6E1AC0EFFF49
:102CC000A82BFCD6FF0ED880C155C26FCE6F000175
:102CD000D5EC0CF0E6EC0CF0E6EC0CF0F5EC0CF0BE
:102CE0001B52D8B44FD11B50E508D8B44BD10301C7
:102CF000A76BA96BA95114080BE3036AA951660FCE
:102D0000E96E030E0320EA6EFF0EEF6EA92BF2D7D9
:102D1000A86BA8C3A7F3A8510A081AE3A751010B8F
:102D2000006EC36BE8B0C38FA751FE0B006ED89046
:102D300000320050C311C56F036AA8511B0FE96E22
:102D4000000E0320EA6EEF50C525A76FA82BE3D72E
:102D5000AB6B4850A75DD8A4FAD03CC066F33EC028
:102D600067F340C068F342C069F344C06AF349C0E6
:102D70006BF34BC06CF34DC06DF34FC06EF351C09D
:102D80006FF353C070F357C071F359C072F30D0E57
:102D9000AB6FA96BA9510C080DE3036AA951660F2B
:102DA000E96E030E0320EA6EEF5202E1A9C3ABF312
:102DB000A92BF0D76850A75DD8A4C8D05CC073F326
:102DC0005EC074F360C075F362C076F364C077F3DD
:102DD00069C078F36BC079F36DC07AF36FC07BF391
:102DE00071C07CF373C07DF377C07EF379C07FF34D
:102DF000190EAB6F0D0EA96FA95119080DE3036AE7
:102E0000A951660FE96E030E0320EA6EEF5202E14C
:102E1000A9C3ABF3A92BF0D7000188510301A75D2B
:102E2000D8A494D07CC080F37EC081F380C082F3AC
:102E300082C083F384C084F389C085F38BC086F39A
:102E40008DC087F38FC088F391C089F393C08AF354
:102E500097C08BF399C08CF3260EAB6F1A0EA96F37
:102E6000A95126080DE3036AA951660FE96E030E06
:102E70000320EA6EEF5202E1A9C3ABF3A92BF0D70E
:102E80000001A8510301A75D2EE19CC08DF39EC0F7
:102E90008EF3A0C08FF3A2C090F3A4C091F3A9C099
:102EA00092F3ABC093F3ADC094F3AFC095F3B1C050
:102EB00096F3B3C097F3B7C098F3B9C099F3330E44
:102EC000AB6F270EA96FA95133080DE3036AA9510F
:102ED000660FE96E030E0320EA6EEF5202E1A9C30A
:102EE000ABF3A92BF0D70001C8510301A75D2EE178
:102EF000BCC09AF3BEC09BF3C0C09CF3C2C09DF39C
:102F0000C4C09EF3C9C09FF3CBC0A0F3CDC0A1F352
:102F1000CFC0A2F3D1C0A3F3D3C0A4F3D7C0A5F30D
:102F2000D9C0A6F3400EAB6F340EA96FA95140086B
:102F30000DE3036AA951660FE96E030E0320EA6EE2
:102F4000EF5202E1A9C3ABF3A92BF0D71AD01BC0F3
:102F500066F31CC067F31DC068F31EC069F31FC091
:102F60006AF320C06BF321C06CF322C06DF32E0E08
:102F70006E6F23C06FF324C070F325C071F30C0E85
:102F8000AB6F00011B5205E1000E016E030116D16B
:102F900000011B50E508D8B40ED123C0ACF324C007
:102FA000ADF325C0AEF30301AC516D0809E0AC519F
:102FB0004D0806E0AC51570803E0AC5177080FE12B
:102FC000AD51500809E0AD51700806E0AD5141081F
:102FD00003E0AD51610803E1AE51330807E0AE51A3
:102FE000560804E0AE517608D8A4E4D0C56B2F5043
:102FF000C525AF6F000E3020B06FB16BB26BB0C3A0
:10300000B2F3AFC3B1F3AF6BB06BC46BC36BC76B41
:103010003550C7250101006F000E03013620010164
:10302000016F000E0301C3210101026F000E0301B5
:10303000C4210101036F0301AF5101010027030106
:10304000B051010101230301B15101010223030128
:10305000B251010103230301C56BC46BC36B35C0BF
:10306000C2F3C96BC86BC76B36C0C6F3C8C303F0E5
:10307000C7C302F036C001F0006A00503524CB6FA0
:103080003650C321CC6FC751C421CD6FC851C52163
:10309000CE6F186AF2BE188EF29EE76FCDC3E6F3CC
:1030A000CCC3E5F3CBC3E4F3EB6BEA6BE96BE3C0B2
:1030B000E8F30001B4EC05F018BEF28EE451030110
:1030C0000024D06F0001E55103010120D16F000EF3
:1030D0000220D26F000E0320D36F0001E6510301DE
:1030E000D0250001EC6FE7510301D1210001ED6F04
:1030F000000E0301D2210001EE6F000E0301D32167
:103100000001EF6F0301C36BF00EE96EC3C3EAFF6A
:1031100037C0EFFFC36BF00EC26F010EC225016E08
:10312000000EC32101C0E9FFEA6E38C0EFFFC36B98
:10313000F00EC26F020EC225016E000EC32101C047
:10314000E9FFEA6E39C0EFFFC36BF00EC26F030EEA
:10315000C225016E000EC32101C0E9FFEA6E3AC02C
:10316000EFFF655324E00D0E000110EC05F00A0E90
:1031700010EC05F00301AA6BAB51AA5D10E2036AE3
:10318000AA51660FE96E030E0320EA6EEFCFC2F379
:10319000C251000110EC05F00301AA2BEDD70D0E72
:1031A000000110EC05F00A0E10EC05F00301010E11
:1031B000016E04D00001000E016E03010001000C3D
:1031C000020E03017E6F7F6B080E806F040E816F0D
:1031D000000181EC08F0010E0301D16F0001B9EC90
:1031E00007F0FF0ED880DD5503017C6FFF0ED880FD
:1031F0000001DC5503017D6F020E7E6F0B0E7F6FA9
:103200007CC380F37DC381F3000181EC08F0010EE3
:103210000301D16F0001B9EC07F0010E0301D16F7A
:103220000001B9EC07F045EF19F08A96100E030182
:103230007E6F7D6B7D5302E17E5312E0886B00014F
:103240004DEC08F0000E81A4010E03017C1503E093
:103250000001F8D703017D51D8B47E077D07EAD776
:103260008A860001000C03017A6B796B786B776BAF
:10327000766B756B020E7E6F0B0E7F6FFE0E806F8E
:10328000816F000181EC08F09BD7FF0ED880DD55DF
:1032900003017C6FFF0ED8800001DC5503017D6FB8
:1032A000020E7E6F0B0E7F6F7CC380F37DC381F3B4
:1032B000000181EC08F003016151655D716F62519D
:1032C0006659726F63516759736F64516859746FAF
:1032D000186AF2BE188EF29E64C3F4F363C3F3F36C
:1032E00062C3F2F361C3F1F3F86BF76BF66BE3C003
:1032F000F5F3000114EC05F018BEF28E03C064F380
:1033000002C063F301C062F300C061F3186AF2BE49
:10331000188EF29E68C3F4F367C3F3F366C3F2F347
:1033200065C3F1F30301F86BF76BF66BE3C0F5F3DC
:10333000000114EC05F018BEF28E03C068F302C061
:1033400067F301C066F300C065F3F28AE1910301FF
:103350007B6B94948B847A6B0001E35103017A5D5B
:10336000D8B08CEF1EF0010E7527D8B0762BD8B4EC
:10337000772BD8B4782B020E0101005D0301696F31
:10338000000E0101015903016A6F000E010102598B
:1033900003016B6F000E0101035903016C6FE3C061
:1033A00000F0016A026A036A03C07FF302C07EF381
:1033B00001C07DF3E3C07CF3186AF2BE188EF29E62
:1033C0006CC3E7F36BC3E6F36AC3E5F369C3E4F3E5
:1033D00003C0EBF302C0EAF301C0E9F3E3C0E8F392
:1033E0000001B4EC05F018BEF28E03C06CF302C00D
:1033F0006BF301C06AF300C069F3FC510301692754
:103400000001FD5103016A230001FE5103016B23FA
:103410000001FF5103016C23016A026A036A7A51B9
:10342000692701506A2302506B2303506C237851A3
:10343000745DD8A06DEF1DF011E17751735DD8A0D8
:103440006DEF1DF00BE17651725DD8A06DEF1DF0B0
:1034500005E17151755DD8B06DEF1DF06CC37FF360
:103460006BC37EF36AC37DF369C37CF34CC3C6FFB1
:10347000D8907C377D377E377F37C950FF0EC96EB5
:10348000C730FEE3C950FF0EC96EC730FEE38B9212
:10349000C950510EC96EC730FEE3030E856F7C0E16
:1034A000846F020E8425016E000E8521036E01C01B
:1034B000E9FFEA6EEFCF86F3C95086C3C9FFC73074
:1034C000FEE3030E856F7C0E846F010E8425016E72
:1034D000000E8521036E01C0E9FFEA6EEFCF86F38F
:1034E000C95086C3C9FFC730FEE3030E856F7C0E4B
:1034F00085C303F0E96E85C3EAFFEFCF86F3C950B9
:1035000086C3C9FFC730FEE3C950C96AC730FEE3AE
:10351000C950FF0EC96EC730FEE3D76B020ED96FDC
:10352000080ED86FD85302E1D95312E0C950FF0EEC
:10353000C96EC730FEE3C9CFDAF3D751DA5D03E1D4
:10354000000E016E07D0D851D8B4D907D807EAD7F2
:10355000010E016E0152D8A475D0FE0ED76F020E77
:10356000D96F080ED86FD85302E1D95312E0C95071
:10357000FF0EC96EC730FEE3C9CFDAF3D751DA5D6B
:1035800003E1000E016E07D0D851D8B4D907D8078F
:10359000EAD7010E016E01523DE18A96816B100E51
:1035A000806F805302E181531AE081B401D0FDD7CE
:1035B0008A9A836B826B83530CE182511F0809E363
:1035C000C950FF0EC96EC730FEE3822BD8B4832BDF
:1035D000F2D78A8A8051D8B481078007E2D78A86D9
:1035E0004CC3C6FFC950FF0EC96EC730FEE3C950B9
:1035F000FF0EC96EC730FEE38B82C950FF0EC96E45
:10360000C730FEE3C950FF0EC96EC730FEE3000E9F
:10361000016E2FD0C950FF0EC96EC730FEE3C950EE
:10362000FF0EC96EC730FEE38B82C950FF0EC96E14
:10363000C730FEE3C950FF0EC96EC730FEE3010E6E
:10364000016E17D0C950FF0EC96EC730FEE3C950D6
:10365000FF0EC96EC730FEE38B82C950FF0EC96EE4
:10366000C730FEE3C950FF0EC96EC730FEE3010E3E
:10367000016E012C32D2210E000110EC05F06CC35A
:103680007FF36BC37EF36AC37DF369C37CF34CC3E2
:10369000C6FFD89003017C377D377E377F37C9500E
:1036A000FF0EC96EC730FEE3C950FF0EC96EC730AA
:1036B000FEE38B92C950510EC96EC730FEE3030E74
:1036C000856F7C0E846F020E8425016E000E8521AD
:1036D000036E01C0E9FFEA6EEFCF86F3C95086C3DF
:1036E000C9FFC730FEE3030E856F7C0E846F010EA9
:1036F0008425016E000E8521036E01C0E9FFEA6E8C
:10370000EFCF86F3C95086C3C9FFC730FEE3030E6F
:10371000856F7C0E85C303F0E96E85C3EAFFEFCFAA
:1037200086F3C95086C3C9FFC730FEE3C950C96AD2
:10373000C730FEE3C950FF0EC96EC730FEE3D76B3A
:10374000020ED96F080ED86FD85302E1D95312E098
:10375000C950FF0EC96EC730FEE3C9CFDAF3D751A7
:10376000DA5D03E1000E016E07D0D851D8B4D90755
:10377000D807EAD7010E016E0152D8A475D0FE0E0B
:10378000D76F020ED96F080ED86FD85302E1D95304
:1037900012E0C950FF0EC96EC730FEE3C9CFDAF39D
:1037A000D751DA5D03E1000E016E07D0D851D8B4CD
:1037B000D907D807EAD7010E016E01523DE18A967A
:1037C000816B100E806F805302E181531AE081B447
:1037D00001D0FDD78A9A836B826B83530CE18251AF
:1037E0001F0809E3C950FF0EC96EC730FEE3822BE4
:1037F000D8B4832BF2D78A8A8051D8B48107800746
:10380000E2D78A864CC3C6FFC950FF0EC96EC730C7
:10381000FEE3C950FF0EC96EC730FEE38B82C9506C
:10382000FF0EC96EC730FEE3C950FF0EC96EC73028
:10383000FEE3000E016E2FD0C950FF0EC96EC730D7
:10384000FEE3C950FF0EC96EC730FEE38B82C9503C
:10385000FF0EC96EC730FEE3C950FF0EC96EC730F8
:10386000FEE3010E016E17D0C950FF0EC96EC730BE
:10387000FEE3C950FF0EC96EC730FEE38B82C9500C
:10388000FF0EC96EC730FEE3C950FF0EC96EC730C8
:10389000FEE3010E016E012C20D1400E000110EC60
:1038A00005F06CC37FF36BC37EF36AC37DF369C31A
:1038B0007CF34CC3C6FFD89003017C377D377E373D
:1038C0007F37C950FF0EC96EC730FEE3C950FF0EE7
:1038D000C96EC730FEE38B92C950510EC96EC73016
:1038E000FEE3030E856F7C0E846F020E8425016E4D
:1038F000000E8521036E01C0E9FFEA6EEFCF86F36B
:10390000C95086C3C9FFC730FEE3030E856F7C0E26
:10391000846F010E8425016E000E8521036E01C0A7
:10392000E9FFEA6EEFCF86F3C95086C3C9FFC730FF
:10393000FEE3030E856F7C0E85C303F0E96E85C33D
:10394000EAFFEFCF86F3C95086C3C9FFC730FEE355
:10395000C950C96AC730FEE3C950FF0EC96EC730EF
:10396000FEE3D76B020ED96F080ED86FD85302E171
:10397000D95312E0C950FF0EC96EC730FEE3C9CF5C
:10398000DAF3D751DA5D03E1000E016E07D0D851AA
:10399000D8B4D907D807EAD7010E016E0152D8A4CE
:1039A00075D0FE0ED76F020ED96F080ED86FD853A0
:1039B00002E1D95312E0C950FF0EC96EC730FEE3D1
:1039C000C9CFDAF3D751DA5D03E1000E016E07D0FB
:1039D000D851D8B4D907D807EAD7010E016E0152E1
:1039E0003DE18A96816B100E806F805302E1815316
:1039F0001AE081B401D0FDD78A9A836B826B83531E
:103A00000CE182511F0809E3C950FF0EC96EC7308F
:103A1000FEE3822BD8B4832BF2D78A8A8051D8B4A4
:103A200081078007E2D78A864CC3C6FFC950FF0EC4
:103A3000C96EC730FEE3C950FF0EC96EC730FEE342
:103A40008B82C950FF0EC96EC730FEE3C950FF0E0E
:103A5000C96EC730FEE3000E016E2FD0C950FF0EB5
:103A6000C96EC730FEE3C950FF0EC96EC730FEE312
:103A70008B82C950FF0EC96EC730FEE3C950FF0EDE
:103A8000C96EC730FEE3010E016E17D0C950FF0E9C
:103A9000C96EC730FEE3C950FF0EC96EC730FEE3E2
:103AA0008B82C950FF0EC96EC730FEE3C950FF0EAE
:103AB000C96EC730FEE3010E016E012C0ED07C6B87
:103AC0007C5100016FEC02F003017C2B000110EC33
:103AD00005F00E0E03017C5DF3E10001DB510708E8
:103AE000D8A4B2D09EAA1DD09EAAFED7AECF7BF39B
:103AF00003017B5175080BE10001DC3D01D001D0D1
:103B0000DC2BDD3D01D001D0DD2B0BD003017B513F
:103B1000640808E10001DC5301E0DC07DD5301E04B
:103B2000DD0703017B51390818E1F29A8B94020EEC
:103B30007E6F0B0E7F6FFE0E806F816F000181EC38
:103B400008F003017C6B000115EC19F0390E10EC44
:103B500005F0390E016EC1D103017B514D0818E10A
:103B6000F29A8B94020E7E6F0B0E7F6FFE0E806FAB
:103B7000816F000181EC08F003017C6B000115EC02
:103B800019F04D0E10EC05F04D0E016EA6D103019B
:103B900083A003D07B516E0815E1F29A8B947C6B65
:103BA000000115EC19F0020E03017E6F0B0E7F6F02
:103BB000FE0E806F816F000181EC08F06E0E016EC9
:103BC0008CD1030183A203D07B5170081FE1000157
:103BD000F45306E1F55304E1F65302E1F75315E01F
:103BE000F29A8B94020E03017E6F0B0E7F6FFE0E16
:103BF000806F816F000181EC08F003017C6B000194
:103C000015EC19F0700E016E68D1030183AA03D080
:103C10007B517A081AE1D00E0001DC6FDD6FF29A59
:103C20008B94020E03017E6F0B0E7F6FFE0E806F72
:103C3000816F000181EC08F003017C6B000115EC41
:103C400019F07A0E016E49D103010001DB5313E133
:103C5000833C01D00FD0E1A50CD0E195F76BF66B5A
:103C6000F56B83CFF4F0E191E1838B946B0E016EE1
:103C700034D101D0E185F5EC10F0E1AB09D00A0EAA
:103C80000301D16F0001B9EC07F0F5EC10F0F5D7A6
:103C9000E02D10D0F29A8B94020E03017E6F0B0E72
:103CA0007F6FFE0E806F816F000181EC08F0650E62
:103CB000016E13D1E1A12CD0F29AE19103017C6B4A
:103CC0007C51000184EC02F003017C2B000110EC1C
:103CD00005F0160E03017C5DF3E10D0E000110EC02
:103CE00005F00A0E10EC05F08B94020E03017E6FB6
:103CF0000B0E7F6FFE0E806F816F000181EC08F06C
:103D000003017C6B000115EC19F06B0E016EE5D020
:103D100003017A2BACEF19F00A0E6525006E000E38
:103D20006621016E000E6721026E000E6821036E8F
:103D30006451035C28E30BE16351025C24E307E177
:103D40006251015C20E303E10050615D1CE203C1AC
:103D500007F102C106F101C105F100C104F107C17B
:103D6000C5F306C1C4F305C1C3F304C1C2F3000126
:103D7000ADEC0FF003C003F102C002F101C001F18C
:103D800000C000F10301FF0ED8800001DD550301E2
:103D90007C6FFF0ED8800001DC5503017D6F020EA1
:103DA0007E6F0B0E7F6F7CC380F37DC381F30001B8
:103DB00081EC08F0DB510708D8A466D083A805D0B1
:103DC00003017B51680861E10001140E0301D16F0A
:103DD0000001B9EC07F083B807D0140E0301D16FCE
:103DE0000001B9EC07F0F7D783A845D09EAA26D0EA
:103DF0009EAAFED7AECF7BF303017B51680806E194
:103E0000300E7B6F000137D019D003017B5175084C
:103E10000BE10001DC3D01D001D0DC2BDD3D01D008
:103E200001D0DD2B0BD003017B51640808E10001B8
:103E3000DC5301E0DC07DD5301E0DD070301140E74
:103E4000D16F0001B9EC07F0E02D14D08B94020E75
:103E500003017E6F0B0E7F6FFE0E806F816F00017E
:103E600081EC08F003017C6B000115EC19F0650E84
:103E7000016E33D0B9D783B801D0FDD7140E03013A
:103E8000D16F0001B9EC07F0030100C16DF301C16E
:103E90006EF302C16FF3010103510F0B0301706F49
:103EA00070510F0814E3D8A4ABEF19F06F51FF085D
:103EB0000EE3D8A4ABEF19F06E51FF0808E3D8A4C5
:103EC000ABEF19F06D51EE08D8B0ABEF19F0F29AE4
:103ED0000001E1938B94730E016E000C0301656B7E
:103EE00002012EAF04D0010E0301656F02012EAB5B
:103EF00004D0010E0301651B02012EA904D0010E9E
:103F00000301651B02012EA504D0010E0301651BF0
:103F10000201D8902E370301655102012E132EC2E3
:103F200001F00001000CFF0E0301606F5F6F0101E3
:103F3000135357E1125355E111510301605DD8B09D
:103F400002D001014ED005E15F510101105D49E24F
:103F50000301010E4827D8B0492BD8B44A2BD8B456
:103F60004B2B0001BBDF010E015C0301616F2E0EC4
:103F70006125E96E010EEA6ED8B0EA2AEF3C01D065
:103F80001DD02E0E6125E96E010EEA6ED8B0EA2A28
:103F9000EF50EF2A626F6251F2CF63F3F29E00019D
:103FA00061EC00F0030163BFF28E606B5F6F61C371
:103FB0005EF35D6B5D515F275E5160234B530AE1F9
:103FC0004A5308E14951FC080AE2FF0A03E148515B
:103FD000E80805E2006A016A026A036A09D0A7D705
:103FE00001015FC300F060C301F0026A036A0301CC
:103FF0000001C4EF27F00301646B110EC26E0A0EBC
:10400000C16EBE0EC06E636B63510F0818E313C11F
:1040100003F012C102F011C101F010C100F06351B0
:10402000656F07E0D8900332023201320032652F0B
:10403000F9D700A002D063C364F3632BE5D7000176
:104040004DDF0301616B01C060F360C361F3606B1E
:10405000000144DF015003016027000E61230000CE
:104060000F0E636F6351645D16E2036A010E026E08
:104070006351006E05E0D89002360336002EFBD760
:104080000250FF0A006EFF0E031A00506017035023
:1040900061176307E7D75F6B5E6B636B6351645DAA
:1040A0002EE3C282C2A201D0FDD7C3A002D062819A
:1040B00001D06291090E006E002EFED700D0C282A0
:1040C000C2A201D0FDD7000EC3B0010E656F000E75
:1040D00062B1010E655D12E062A10FD0036A010EAC
:1040E000026E6351006E05E0D89002360336002E52
:1040F000FBD702505E1303505F13632BCFD7605181
:104100005E1B61515F1B0101135311E112530FE15B
:10411000115103015F5DD8B002D0010108D009E15F
:104120005E510101105DD8B002D0030102D0000E33
:1041300001D0010E03015D1582E12E0E000110EC8D
:1041400005F0010EC26E03015EC301F05FC302F011
:104150000001D6EF27F0F86AD09E088EFE0E006EA2
:10416000040E016E020EE96E000EEA6EEE6A002E7B
:10417000FDD7012EFBD7EA6AE96AB886110EAF6E49
:10418000040EB06EA60EAC6E900EAB6EC150C00B9E
:104190000F09C16E070EB46EE26B8B6A7F0E926ED2
:1041A000C50E936E940E946EFF0E956E070E966E6E
:1041B0009B8C010EC26E94948B940F0EC16E80CFB7
:1041C000DBF0070EDB1780A604D0220E03014C6F34
:1041D00003D0200E03014C6F0A0EC16E880EC06E14
:1041E000F19CF19EF292820ED56E8B808A92320EF5
:1041F000D16F0001B9EC07F00D0E10EC05F00A0EBE
:1042000010EC05F00D0E10EC05F00A0E10EC05F0A8
:1042100003015D6B0001CEEF07F00D0E10EC05F011
:104220000A0E10EC05F00D0E10EC05F00A0E10EC65
:1042300005F003015D6B5D510001EEEC00F0030140
:104240005D2B000110EC05F03C0E03015D5DF3E118
:104250000D0E000110EC05F00A0E10EC05F00D0E2D
:1042600010EC05F00A0E10EC05F08B828A888A8625
:10427000C69A320E0301D16F0001B9EC07F08A92A1
:10428000FA0E03015D6F00013AEF08F08A82320EE8
:104290000301D16F0001B9EC07F0320E0301D16FB9
:1042A0000001B9EC07F081A4EAD7A60E006E002E3B
:1042B000FED70000020E03017E6F7F6B806B040E41
:1042C000816F000181EC08F00A0E0301D16F00013B
:1042D000B9EC07F081A4E9D7320E0301D16F0001D8
:1042E000B9EC07F0320E0301D16F0001B9EC07F011
:1042F00081A4F2D7010E0301D16F0001B9EC07F0E0
:10430000020E03017E6F7F6B080E806F816B0001D0
:1043100081EC08F0FF0ED880DD5503015D6FFF0EC4
:10432000D8800001DC5503015E6F020E7E6F0B0E1C
:104330007F6F5DC380F35EC381F3000181EC08F001
:10434000010E0301D16F0001B9EC07F003015D6BB1
:104350005D51000178EC03F0000907E003015D2BDB
:104360009EA8FED7AD6EF4D700010D0E9EA8FED715
:10437000AD6E0A0E9EA8FED7AD6E8A888A86E19B36
:10438000E06BDF6BDF0EDD6FDC6F03014D6B000157
:10439000E19DE19F03014E91536B300E0001DE6FF2
:1043A000010E0301506F516B502D01D002D0000E51
:1043B00001D0010E5D6F5151090802E2000E01D0DB
:1043C000010E5D150AE0010ECD6F000118EC09F039
:1043D00001C050F30301512BE7D7502D10D05D6B76
:1043E0005D5100011AEC01F003015D2B000110EC9E
:1043F00005F0290E03015D5DF3E10300FED7000126
:104400002EEC0DF0EA5303E1EB51020818E0030132
:104410005D6B5D5100013CEC01F003015D2B00017F
:1044200010EC05F0130E03015D5DF3E10D0E0001CC
:1044300010EC05F00A0E10EC05F02EEC0DF0030167
:104440005D6B5D51000153EC01F003015D2B000138
:1044500010EC05F0110E03015D5DF3E10D0E00019E
:1044600010EC05F00A0E10EC05F0F76BF66BF56B2F
:10447000010EF46F70EF10F003015D6B5D510001F0
:1044800069EC01F003015D2B000110EC05F0110E49
:1044900003015D5DF3E110C1D1F31B0ED26F00018A
:1044A000D9EC08F00D0E10EC05F00A0E10EC05F03A
:1044B0001BC10BF11AC10AF119C109F118C108F1A8
:1044C000730E03014F6F0001E199E1830301506B0B
:1044D0000001E191E197C00EF212F29A010113532B
:1044E0000AE1125308E1115100080AE2FF0A03E150
:1044F0001051180805E28C0E0301476F09D0010125
:10450000D8901331123111311031E8CF47F3030144
:10451000516B4751515D11E2D8905135026E036ADB
:10452000033602502F0FE96E020E0320EA6EFF0ED3
:10453000EC6EED52EF6E512BECD70D0E000110EC2E
:1045400005F00A0E10EC05F00D0E10EC05F00A0E49
:1045500010EC05F003014C5120080FE15D6B5D513B
:10456000000180EC01F003015D2B000110EC05F06F
:10457000390E03015D5DF3E10ED05D6B5D5100010D
:10458000AAEC01F003015D2B000110EC05F0120E06
:1045900003015D5DF3E10D0E000110EC05F00A0E64
:1045A00010EC05F0F5EC10F0DB510608D8A45AD158
:1045B0009D8A0D0E10EC05F00A0E10EC05F00301BB
:1045C0005D6B5D510001C1EC01F003015D2B000149
:1045D00010EC05F0190E03015D5DF3E10D0E000115
:1045E00010EC05F00A0E10EC05F00D0E10EC05F0C5
:1045F0000A0E10EC05F0010EDF6FE193F76BF66B1E
:10460000FF0EF56FF46FF5C05EF3F4C05DF3F5C017
:1046100060F3F4C05FF32BEC11F003C058F302C059
:1046200057F301C056F300C055F3E1B90CD0E1B324
:104630000AD0640E0301D16F0001B9EC07F02E0E11
:1046400010EC05F0F2D7F5C05EF3F4C05DF3F5C0F1
:1046500060F3F4C05FF32BEC11F003C058F302C019
:1046600057F301C056F300C055F30301555307E15A
:10467000565305E1575303E15853D8B4F1D058537A
:1046800007E1575305E1565303E15551040818E279
:10469000050E555D5D6F000E56595E6F000E575941
:1046A0005F6F000E5859606F646F5FC363F35EC342
:1046B00062F35DC361F3656B000141EC14F003012B
:1046C000585307E1575305E1565303E15551030889
:1046D00018E2040E555D5D6F000E56595E6F000EB8
:1046E00057595F6F000E5859606F646F5FC363F373
:1046F0005EC362F35DC361F3656B000141EC14F0CE
:104700000301585307E1575305E1565303E155514F
:10471000020818E2030E555D5D6F000E56595E6F7C
:10472000000E57595F6F000E5859606F646F5FC37A
:1047300063F35EC362F35DC361F3656B000141EC3B
:1047400014F00301585307E1575305E1565303E1B1
:104750005551010818E2020E555D5D6F000E565965
:104760005E6F000E57595F6F000E5859606F646F8F
:104770005FC363F35EC362F35DC361F3656B000106
:1047800041EC14F00301555306E1565304E157532D
:1047900002E1585318E0010E555D5D6F000E565949
:1047A0005E6F000E57595F6F000E5859606F646F4F
:1047B0005FC363F35EC362F35DC361F3656B0001C6
:1047C00041EC14F0030158C364F357C363F356C3B9
:1047D00062F355C361F3010E656F000141EC14F003
:1047E0000D0E10EC05F00A0E10EC05F0D890036ADF
:1047F000F331026EF231016EF131006EEC250301EE
:104800005D6F01500001ED2103015E6F0250000158
:10481000EE2103015F6F03500001EF210301606F80
:10482000EFC064F3EEC063F3EDC062F3ECC061F37C
:10483000686F5FC367F35EC366F35DC365F3000132
:1048400033EC19F001C04FF3E1A904D0E1B302D079
:10485000030115D7010E0301D16F0001B9EC07F078
:104860000001E3D6DB53D8A407D103015D6B5D5192
:104870000001DBEC01F003015D2B000110EC05F001
:10488000130E03015D5DF3E10D0E000110EC05F068
:104890000A0E10EC05F0E193010EDF6FE1B305D0D5
:1048A000F76BF66BF56B83CFF4F00301586B576B26
:1048B000566B556B0001F451FE080CE1F5530AE10B
:1048C000F65308E1F75306E103015C6B5B6B5A6B2F
:1048D000596B0001F451FD080DE1F5530BE1F6535E
:1048E00009E1F75307E103015C6B5B6B5A6B010E47
:1048F000596F0001F451FB080DE1F5530BE1F6533C
:1049000009E1F75307E103015C6B5B6B5A6B020E25
:10491000596F0001F451F7080DE1F5530BE1F6531F
:1049200009E1F75307E103015C6B5B6B5A6B030E04
:10493000596F0001F451EF080DE1F5530BE1F65307
:1049400009E1F75307E103015C6B5B6B5A6B040EE3
:10495000596F0001F451DF080DE1F5530BE1F653F7
:1049600009E1F75307E103015C6B5B6B5A6B050EC2
:10497000596F0001F451BF080DE1F5530BE1F653F7
:1049800009E1F75307E103015C6B5B6B5A6B060EA1
:10499000596F0001F4517F080DE1F5530BE1F65317
:1049A00009E1F75307E103015C6B5B6B5A6B070E80
:1049B000596F0001F43D06D0F55304E1F65302E1CE
:1049C000F75312E05AC35EF359C35DF35AC360F361
:1049D00059C35FF32BEC11F003C058F302C057F337
:1049E00001C056F300C055F30301555306E1565379
:1049F00004E1575302E158533CE058C364F357C3F2
:104A000063F356C362F355C361F3656B000141EC78
:104A100014F0E193D890036AF331026EF231016E23
:104A2000F131006EEC2503015D6F01500001ED21B5
:104A300003015E6F02500001EE2103015F6F03501E
:104A40000001EF210301606FEFC064F3EEC063F378
:104A5000EDC062F3ECC061F3686F5FC367F35EC3E0
:104A600066F35DC365F3000133EC19F001C04FF349
:104A700002D00001E19310D7DB2D1ED103015D6B45
:104A80005D510001F2EC01F003015D2B000110EC1F
:104A900005F0110E03015D5DF3E10D0E000110EC58
:104AA00005F00A0E10EC05F0F288F28A010EDF6FB5
:104AB000E1B701D0FDD7F5C05EF3F4C05DF3F5C0FA
:104AC00060F3F4C05FF32BEC11F003C058F302C0A5
:104AD00057F301C056F300C055F30301555307E1E6
:104AE000565305E1575303E15853D8B4DFD0585318
:104AF00007E1575305E1565303E15551040818E205
:104B0000050E555D5D6F000E56595E6F000E5759CC
:104B10005F6F000E5859606F646F5FC363F35EC3CD
:104B200062F35DC361F3656B000141EC14F00301B6
:104B3000585307E1575305E1565303E15551030814
:104B400018E2040E555D5D6F000E56595E6F000E43
:104B500057595F6F000E5859606F646F5FC363F3FE
:104B60005EC362F35DC361F3656B000141EC14F059
:104B70000301585307E1575305E1565303E15551DB
:104B8000020818E2030E555D5D6F000E56595E6F08
:104B9000000E57595F6F000E5859606F646F5FC306
:104BA00063F35EC362F35DC361F3656B000141ECC7
:104BB00014F00301585307E1575305E1565303E13D
:104BC0005551010818E2020E555D5D6F000E5659F1
:104BD0005E6F000E57595F6F000E5859606F646F1B
:104BE0005FC363F35EC362F35DC361F3656B000192
:104BF00041EC14F00301555306E1565304E15753B9
:104C000002E1585318E0010E555D5D6F000E5659D4
:104C10005E6F000E57595F6F000E5859606F646FDA
:104C20005FC363F35EC362F35DC361F3656B000151
:104C300041EC14F0030158C364F357C363F356C344
:104C400062F355C361F3010E656F000141EC14F08E
:104C5000D890036AF331026EF231016EF131006EC9
:104C6000EC2503015D6F01500001ED2103015E6F32
:104C700002500001EE2103015F6F03500001EF219C
:104C80000301606FEFC064F3EEC063F3EDC062F345
:104C9000ECC061F3686F5FC367F35EC366F35DC327
:104CA00065F3000133EC19F001C04FF30001E1B7E7
:104CB00001D0FDD7E197FFD6DB510408D8A41ED15F
:104CC00003015D6B5D51000108EC02F003015D2BF7
:104CD000000110EC05F0150E03015D5DF3E10D0E12
:104CE000000110EC05F00A0E10EC05F0F288F28AD3
:104CF000010EDF6FE1B701D0FDD7F5C05EF3F4C060
:104D00005DF3F5C060F3F4C05FF32BEC11F003C06A
:104D100058F302C057F301C056F300C055F3030126
:104D2000555307E1565305E1575303E15853D8B49F
:104D3000DFD0585307E1575305E1565303E155516E
:104D4000040818E2050E555D5D6F000E56595E6F42
:104D5000000E57595F6F000E5859606F646F5FC344
:104D600063F35EC362F35DC361F3656B000141EC05
:104D700014F00301585307E1575305E1565303E17B
:104D80005551030818E2040E555D5D6F000E56592B
:104D90005E6F000E57595F6F000E5859606F646F59
:104DA0005FC363F35EC362F35DC361F3656B0001D0
:104DB00041EC14F00301585307E1575305E15653F2
:104DC00003E15551020818E2030E555D5D6F000EB8
:104DD00056595E6F000E57595F6F000E5859606F3D
:104DE000646F5FC363F35EC362F35DC361F3656BBE
:104DF000000141EC14F00301585307E1575305E15A
:104E0000565303E15551010818E2020E555D5D6FDE
:104E1000000E56595E6F000E57595F6F000E5859BD
:104E2000606F646F5FC363F35EC362F35DC361F37E
:104E3000656B000141EC14F00301555306E1565334
:104E400004E1575302E1585318E0010E555D5D6FC0
:104E5000000E56595E6F000E57595F6F000E58597D
:104E6000606F646F5FC363F35EC362F35DC361F33E
:104E7000656B000141EC14F0030158C364F357C3A0
:104E800063F356C362F355C361F3010E656F00010E
:104E900041EC14F0D890036AF331026EF231016EE6
:104EA000F131006EEC2503015D6F01500001ED2131
:104EB00003015E6F02500001EE2103015F6F03509A
:104EC0000001EF210301606FEFC064F3EEC063F3F4
:104ED000EDC062F3ECC061F3686F5FC367F35EC35C
:104EE00066F35DC365F3000133EC19F001C04FF3C5
:104EF0000001E1B701D0FDD7E197FFD6DB510508EE
:104F0000D8A4E0D184B001D0E18D03015D6B5D5187
:104F1000000120EC02F003015D2B000110EC05F014
:104F2000160E03015D5DF3E10D0E000110EC05F0BE
:104F30000A0E10EC05F084B203D081A001D0FDD799
:104F400003014B6B4A6B496B486B020E0001DF6F2C
:104F5000F2880301516B513D01D00AD02E0E51252C
:104F6000E96E010EEA6ED8B0EA2AEF6A512BF3D748
:104F700002012D6BEB0E2E6F170E01011D6F84B415
:104F80000FD0000193EF1FF003C0F7F002C0F6F05E
:104F900001C0F5F000C0F4F00301548132D00101EA
:104FA000010E03015D6F0001FBEF1FF0F76BF66B65
:104FB00002C0F5F001C0F4F00301526B4751525D9D
:104FC00020E2D8905235026E036A033602502F0F4A
:104FD000E96E020E0320EA6EECCF5EF3ED52EFCFE6
:104FE0005DF30001F45103015D5D08E10001F5513D
:104FF00003015E5D03E1549104D001D05481522B32
:10500000DDD754A14DD10001F75307E1F65305E177
:10501000F55303E1F45104081EE2050EF45D0301AB
:105020005D6F000E0001F55903015E6F000E000177
:10503000F65903015F6F000E0001F7590301606F1D
:10504000646F5FC363F35EC362F35DC361F3656B5B
:10505000000141EC14F0F75307E1F65305E1F55375
:1050600003E1F45103081EE2040EF45D03015D6FD9
:10507000000E0001F55903015E6F000E0001F659A4
:1050800003015F6F000E0001F7590301606F646F49
:105090005FC363F35EC362F35DC361F3656B0001DD
:1050A00041EC14F0F75307E1F65305E1F55303E142
:1050B000F45102081EE2030EF45D03015D6F000E61
:1050C0000001F55903015E6F000E0001F65903015E
:1050D0005F6F000E0001F7590301606F646F5FC3DB
:1050E00063F35EC362F35DC361F3656B000141EC82
:1050F00014F0F75307E1F65305E1F55303E1F451DA
:1051000001081EE2020EF45D03015D6F000E000156
:10511000F55903015E6F000E0001F65903015F6F40
:10512000000E0001F7590301606F646F5FC363F302
:105130005EC362F35DC361F3656B000141EC14F083
:10514000F45306E1F55304E1F65302E1F7531EE090
:10515000010EF45D03015D6F000E0001F5590301BE
:105160005E6F000E0001F65903015F6F000E000133
:10517000F7590301606F646F5FC363F35EC362F34B
:105180005DC361F3656B000141EC14F0F7C064F39B
:10519000F6C063F3F5C062F3F4C061F3010E0301DE
:1051A000656F000141EC14F001C050F30301502D74
:1051B0003BD0D890036A0001F331026EF231016EE8
:1051C000F131006EEC2503015D6F01500001ED210E
:1051D00003015E6F02500001EE2103015F6F035077
:1051E0000001EF210301606FEFC064F3EEC063F3D1
:1051F000EDC062F3ECC061F3686F5FC367F35EC339
:1052000066F35DC365F3000133EC19F001C04FF3A1
:1052100084B20BD003014F517308D8B402D00001FF
:1052200004D081A001D0FDD7000184A435D0020EA6
:105230000301475D526F4751525D29E2010E52252D
:10524000036A026ED8900236033602502F0F016EA9
:10525000020E032203C05FF3D8905235026E036A38
:10526000033602502F0FE96E020E0320EA6EECCFD8
:1052700003F0ED52EFCF60F35FC3EAFF01C0E9FF37
:1052800003C0ECFFED5260C3EFFF5207D4D7F5C067
:1052900030F2F4C02FF200013B0E10EC05F00301D8
:1052A0004B530FE14A530DE14951FD080AE3D8B4CD
:1052B00002D0010164D64851E608D8A002D001010D
:1052C0005ED63FD603015D6B5D51000139EC02F003
:1052D00003015D2B000110EC05F00F0E03015D5D75
:1052E000F3E10D0E000110EC05F00A0E10EC05F0D4
:1052F00084B214D09EAA07D09EAAFED7AECF53F395
:1053000003010DD0000183B003D0030108D00001D8
:1053100083B203D0030103D00001ECD7030184B0B2
:1053200003D00001E18D030183B048D0780E516FA6
:1053300051530DE0030ED16F0001B9EC07F083A0CB
:1053400003D0030104D0000103015107F1D783B05A
:1053500035D0010ED16F0001B9EC07F00301512BDC
:1053600051511E082AE1516B010E0001F427D8B0FB
:10537000F52BD8B4F62BD8B4F72B0101135100014B
:10538000F75D1AE314E1010112510001F65D14E327
:105390000EE1010111510001F55D0EE308E1F45148
:1053A0000101105DD8A002D0000106D00001F76B0A
:1053B000F66BF56B010EF46F0301C9D783B239D0D8
:1053C000780E516F51530DE0030ED16F0001B9EC0F
:1053D00007F083A203D0030104D0000103015107A9
:1053E000F1D783B226D0010ED16F0001B9EC07F0DE
:1053F0000301512B51511E081BE1516BFF0E00019F
:10540000F427D8A0F527D8A0F627D8A0F727F4537B
:105410000EE1F5530CE1F6530AE1F75308E113C12D
:10542000F7F012C1F6F011C1F5F010C1F4F003016C
:10543000D8D79EAA04D09EAAFED7AECF53F353511D
:105440006E082BE1010E0001F427D8B0F52BD8B47B
:10545000F62BD8B4F72B010113510001F75D1AE3C5
:1054600014E1010112510001F65D14E30EE10101A6
:1054700011510001F55D0EE308E1F4510101105DE9
:10548000D8A002D0000106D00001F76BF66BF56BD7
:10549000010EF46F0301536B50D0535170081CE19F
:1054A000FF0E0001F427D8A0F527D8A0F627D8A032
:1054B000F727F4530EE1F5530CE1F6530AE1F753E5
:1054C00008E113C1F7F012C1F6F011C1F5F010C1F7
:1054D000F4F00301536B31D0535175080BE1000117
:1054E000DC3D01D001D0DC2BDD3D01D001D0DD2B36
:1054F00025D003015351640809E10001DC5301E0A8
:10550000DC07DD5301E0DD0719D0030153513908F1
:1055100009E10001F76BF66BF56B090EF46F0301FF
:10552000536B0BD053514D0808E10001F76BF66B3C
:10553000F56B200EF46F0301536B000183A0A2D121
:1055400083A2A0D10301516BF7C064F3F6C063F3EB
:10555000F5C062F3F4C061F3656B000141EC14F037
:1055600001C050F30301505102080AE10001F76B3A
:10557000F66BF56B010EF46F730E03014F6F2AD1BA
:10558000502D28D10001F75307E1F65305E1F553FB
:1055900003E1F45104081EE2050EF45D03015D6FA2
:1055A000000E0001F55903015E6F000E0001F6596F
:1055B00003015F6F000E0001F7590301606F646F14
:1055C0005FC363F35EC362F35DC361F3656B0001A8
:1055D00041EC14F0F75307E1F65305E1F55303E10D
:1055E000F45103081EE2040EF45D03015D6F000E2A
:1055F0000001F55903015E6F000E0001F659030129
:105600005F6F000E0001F7590301606F646F5FC3A5
:1056100063F35EC362F35DC361F3656B000141EC4C
:1056200014F0F75307E1F65305E1F55303E1F451A4
:1056300002081EE2030EF45D03015D6F000E00011F
:10564000F55903015E6F000E0001F65903015F6F0B
:10565000000E0001F7590301606F646F5FC363F3CD
:105660005EC362F35DC361F3656B000141EC14F04E
:10567000F75307E1F65305E1F55303E1F45101084F
:105680001EE2020EF45D03015D6F000E0001F5598C
:1056900003015E6F000E0001F65903015F6F000EFB
:1056A0000001F7590301606F646F5FC363F35EC36A
:1056B00062F35DC361F3656B000141EC14F0F453D8
:1056C00006E1F55304E1F65302E1F7531EE0010E43
:1056D000F45D03015D6F000E0001F55903015E6F7B
:1056E000000E0001F65903015F6F000E0001F7592B
:1056F0000301606F646F5FC363F35EC362F35DC3F6
:1057000061F3656B000141EC14F0F7C064F3F6C07F
:1057100063F3F5C062F3F4C061F3010E0301656F3A
:10572000000141EC14F0D890036AF331026EF231BB
:10573000016EF131006EEC2503015D6F0150000137
:10574000ED2103015E6F02500001EE2103015F6F46
:1057500003500001EF210301606FEFC064F3EEC05E
:1057600063F3EDC062F3ECC061F3686F5FC367F38E
:105770005EC366F35DC365F3000133EC19F001C04D
:105780004FF384B228D003014F517308D8B402D02C
:10579000000121D09EAA13D09EAAFED7AECF53F30C
:1057A00019D05D6B5D5100014EEC02F003015D2BE1
:1057B000000110EC05F00A0E03015D5DF3E183B01A
:1057C00003D0730E4F6F06D083B203D0700E4F6FAD
:1057D00001D0E0D7000103014F516E0803E04F51A3
:1057E00073080BE1010E0001F427D8B0F52BD8B4F3
:1057F000F62BD8B4F72B46D003014F517A080AE1B3
:105800000001F76BF66BF56B010EF46F730E03017D
:105810004F6F39D04F5139080AE10001F76BF66B31
:10582000F56B090EF46F730E03014F6F2CD04F51BF
:105830004D080AE10001F76BF66BF56B200EF46F73
:10584000730E03014F6F1FD04F5170081CE1000110
:10585000F75307E1F65305E1F55303E1F45101086D
:1058600009E2FF0EF427D8A0F527D8A0F627D8A084
:10587000F72708D013C1F7F012C1F6F011C1F5F007
:0A58800010C1F4F0030150D503003D
:087FF800A0F4C5FF00F1000038
:00000001FF
